BL51 BANKED LINKER/LOCATER V6.22                                                        04/19/2018  15:13:34  PAGE 1


BL51 BANKED LINKER/LOCATER V6.22, INVOKED BY:
D:\KEIL_51\C51\BIN\BL51.EXE STARTUP.obj, main.obj, oled.obj TO OLED RAMSIZE (256)


MEMORY MODEL: SMALL


INPUT MODULES INCLUDED:
  STARTUP.obj (?C_STARTUP)
  main.obj (MAIN)
  oled.obj (OLED)
  D:\KEIL_51\C51\LIB\C51S.LIB (?C?CLDOPTR)
  D:\KEIL_51\C51\LIB\C51S.LIB (?C?IMUL)
  D:\KEIL_51\C51\LIB\C51S.LIB (?C?UIDIV)
  D:\KEIL_51\C51\LIB\C51S.LIB (?C?OFFXADD)


LINK MAP OF MODULE:  OLED (?C_STARTUP)


            TYPE    BASE      LENGTH    RELOCATION   SEGMENT NAME
            -----------------------------------------------------

            * * * * * * *   D A T A   M E M O R Y   * * * * * * *
            REG     0000H     0008H     ABSOLUTE     "REG BANK 0"
            DATA    0008H     000CH     UNIT         _DATA_GROUP_
            DATA    0014H     0009H     UNIT         ?DT?_OLED_SHOWNUM?OLED
            DATA    001DH     0001H     UNIT         ?DT?_OLED_POW?OLED
            IDATA   001EH     0001H     UNIT         ?STACK

            * * * * * * *   C O D E   M E M O R Y   * * * * * * *
            CODE    0000H     0003H     ABSOLUTE     
            CODE    0003H     3232H     UNIT         ?CO?MAIN
            CODE    3235H     09D8H     UNIT         ?CO?OLED
            CODE    3C0DH     016AH     UNIT         ?PR?_OLED_SHOWCHAR?OLED
            CODE    3D77H     014CH     UNIT         ?PR?_OLED_SHOWCHINESE?OLED
            CODE    3EC3H     00B8H     UNIT         ?PR?MAIN?MAIN
            CODE    3F7BH     00A0H     UNIT         ?C?LIB_CODE
            CODE    401BH     009CH     UNIT         ?PR?INITIAL_SSD1327?OLED
            CODE    40B7H     007EH     UNIT         ?PR?_OLED_DRAWBMP?OLED
            CODE    4135H     0075H     UNIT         ?PR?_OLED_SHOWNUM?OLED
            CODE    41AAH     0031H     UNIT         ?PR?_OLED_SHOWSTRING?OLED
            CODE    41DBH     002AH     UNIT         ?PR?RAINBOW?OLED
            CODE    4205H     0026H     UNIT         ?PR?_WRITE_REGISTER?OLED
            CODE    422BH     0022H     UNIT         ?PR?_CLEARLED?OLED
            CODE    424DH     0021H     UNIT         ?PR?_WRITE_PARAMETER?OLED
            CODE    426EH     001EH     UNIT         ?PR?_DELAY?OLED
            CODE    428CH     0018H     UNIT         ?PR?_OLED_POW?OLED
            CODE    42A4H     0015H     UNIT         ?PR?_COLUMN_ADDRESS?OLED
            CODE    42B9H     0011H     UNIT         ?PR?_ROW_ADDRESS?OLED
            CODE    42CAH     0011H     UNIT         ?PR?_SET_COLUME_ADDRESS?OLED
            CODE    42DBH     0011H     UNIT         ?PR?_SET_ROW_ADDRESS?OLED
            CODE    42ECH     000CH     UNIT         ?C_C51STARTUP
            CODE    42F8H     000AH     UNIT         ?PR?OPEN_DC_POWER?OLED
            CODE    4302H     000AH     UNIT         ?PR?OFF_DC_POWER?OLED



BL51 BANKED LINKER/LOCATER V6.22                                                      04/19/2018  15:13:34  PAGE 2


OVERLAY MAP OF MODULE:   OLED (?C_STARTUP)


SEGMENT                                DATA_GROUP 
  +--> CALLED SEGMENT                START    LENGTH
----------------------------------------------------
?C_C51STARTUP                        -----    -----
  +--> ?PR?MAIN?MAIN

?PR?MAIN?MAIN                        0008H    0001H
  +--> ?PR?INITIAL_SSD1327?OLED
  +--> ?PR?_CLEARLED?OLED
  +--> ?PR?OPEN_DC_POWER?OLED
  +--> ?PR?_OLED_SHOWCHINESE?OLED
  +--> ?CO?MAIN
  +--> ?PR?_OLED_SHOWSTRING?OLED
  +--> ?PR?_OLED_DRAWBMP?OLED
  +--> ?PR?_DELAY?OLED
  +--> ?PR?RAINBOW?OLED

?PR?INITIAL_SSD1327?OLED             -----    -----
  +--> ?PR?_DELAY?OLED
  +--> ?PR?_WRITE_REGISTER?OLED

?PR?_CLEARLED?OLED                   0009H    0001H
  +--> ?PR?_SET_COLUME_ADDRESS?OLED
  +--> ?PR?_SET_ROW_ADDRESS?OLED
  +--> ?PR?_WRITE_PARAMETER?OLED

?PR?_SET_COLUME_ADDRESS?OLED         -----    -----
  +--> ?PR?_WRITE_REGISTER?OLED

?PR?_SET_ROW_ADDRESS?OLED            -----    -----
  +--> ?PR?_WRITE_REGISTER?OLED

?PR?OPEN_DC_POWER?OLED               -----    -----
  +--> ?PR?_WRITE_REGISTER?OLED

?PR?_OLED_SHOWCHINESE?OLED           0009H    0007H
  +--> ?PR?_SET_COLUME_ADDRESS?OLED
  +--> ?PR?_SET_ROW_ADDRESS?OLED
  +--> ?CO?OLED
  +--> ?PR?_WRITE_PARAMETER?OLED

?PR?_OLED_SHOWSTRING?OLED            0009H    0006H
  +--> ?PR?_OLED_SHOWCHAR?OLED

?PR?_OLED_SHOWCHAR?OLED              000FH    0005H
  +--> ?PR?_SET_COLUME_ADDRESS?OLED
  +--> ?PR?_SET_ROW_ADDRESS?OLED
  +--> ?CO?OLED
  +--> ?PR?_WRITE_PARAMETER?OLED

?PR?_OLED_DRAWBMP?OLED               0009H    000BH
  +--> ?PR?_SET_COLUME_ADDRESS?OLED
  +--> ?PR?_SET_ROW_ADDRESS?OLED
  +--> ?PR?_WRITE_PARAMETER?OLED
BL51 BANKED LINKER/LOCATER V6.22                                                      04/19/2018  15:13:34  PAGE 3



?PR?RAINBOW?OLED                     -----    -----
  +--> ?PR?_SET_COLUME_ADDRESS?OLED
  +--> ?PR?_SET_ROW_ADDRESS?OLED
  +--> ?PR?_WRITE_PARAMETER?OLED



SYMBOL TABLE OF MODULE:  OLED (?C_STARTUP)

  VALUE           TYPE          NAME
  ----------------------------------

  -------         MODULE        ?C_STARTUP
  C:42ECH         SEGMENT       ?C_C51STARTUP
  I:001EH         SEGMENT       ?STACK
  C:0000H         PUBLIC        ?C_STARTUP
  D:00E0H         SYMBOL        ACC
  D:00F0H         SYMBOL        B
  D:0083H         SYMBOL        DPH
  D:0082H         SYMBOL        DPL
  N:0000H         SYMBOL        IBPSTACK
  N:0100H         SYMBOL        IBPSTACKTOP
  N:0080H         SYMBOL        IDATALEN
  C:42EFH         SYMBOL        IDATALOOP
  N:0000H         SYMBOL        PBPSTACK
  N:0100H         SYMBOL        PBPSTACKTOP
  N:0000H         SYMBOL        PDATALEN
  N:0000H         SYMBOL        PDATASTART
  N:0000H         SYMBOL        PPAGE
  N:0000H         SYMBOL        PPAGEENABLE
  D:00A0H         SYMBOL        PPAGE_SFR
  D:0081H         SYMBOL        SP
  C:42ECH         SYMBOL        STARTUP1
  N:0000H         SYMBOL        XBPSTACK
  N:0000H         SYMBOL        XBPSTACKTOP
  N:0000H         SYMBOL        XDATALEN
  N:0000H         SYMBOL        XDATASTART
  C:0000H         LINE#         126
  C:42ECH         LINE#         133
  C:42EEH         LINE#         134
  C:42EFH         LINE#         135
  C:42F0H         LINE#         136
  C:42F2H         LINE#         185
  C:42F5H         LINE#         196
  -------         ENDMOD        ?C_STARTUP

  -------         MODULE        MAIN
  C:0000H         SYMBOL        _ICE_DUMMY_
  D:0090H         PUBLIC        P1
  C:1235H         PUBLIC        BMP2
  C:3EC3H         PUBLIC        main
  C:0035H         PUBLIC        BMP
  -------         PROC          MAIN
  -------         DO            
  D:0008H         SYMBOL        t
  -------         ENDDO         
BL51 BANKED LINKER/LOCATER V6.22                                                      04/19/2018  15:13:34  PAGE 4


  C:3EC3H         LINE#         34
  C:3EC3H         LINE#         35
  C:3EC3H         LINE#         36
  C:3EC6H         LINE#         39
  C:3EC6H         LINE#         40
  C:3EC6H         LINE#         42
  C:3ECBH         LINE#         43
  C:3ECEH         LINE#         44
  C:3ED6H         LINE#         45
  C:3EDFH         LINE#         46
  C:3EE8H         LINE#         47
  C:3EF1H         LINE#         48
  C:3EFAH         LINE#         49
  C:3F03H         LINE#         50
  C:3F0CH         LINE#         52
  C:3F19H         LINE#         53
  C:3F26H         LINE#         54
  C:3F33H         LINE#         57
  C:3F47H         LINE#         60
  C:3F4EH         LINE#         61
  C:3F53H         LINE#         62
  C:3F67H         LINE#         64
  C:3F6EH         LINE#         65
  C:3F71H         LINE#         66
  C:3F78H         LINE#         67
  -------         ENDPROC       MAIN
  -------         ENDMOD        MAIN

  -------         MODULE        OLED
  C:0000H         SYMBOL        _ICE_DUMMY_
  B:0090H.2       PUBLIC        OLED_RST
  D:0090H         PUBLIC        P1
  C:42F8H         PUBLIC        OPEN_DC_POWER
  C:424DH         PUBLIC        _Write_Parameter
  B:0090H.4       PUBLIC        OLED_CS
  C:42A4H         PUBLIC        _Column_Address
  C:42CAH         PUBLIC        _Set_Colume_Address
  C:41AAH         PUBLIC        _OLED_ShowString
  C:3C0DH         PUBLIC        _OLED_ShowChar
  B:0090H.3       PUBLIC        OLED_RS
  C:3235H         PUBLIC        F6x8
  C:3A4DH         PUBLIC        Hzk
  C:4302H         PUBLIC        OFF_DC_POWER
  B:0090H.1       PUBLIC        OLED_SDIN
  C:420AH         PUBLIC        _Write_Register
  C:345DH         PUBLIC        F8X16
  C:422BH         PUBLIC        _ClearLED
  C:401BH         PUBLIC        Initial_ssd1327
  C:3D77H         PUBLIC        _OLED_ShowCHinese
  C:41DBH         PUBLIC        Rainbow
  C:4135H         PUBLIC        _OLED_ShowNum
  C:428CH         PUBLIC        _oled_pow
  C:42B9H         PUBLIC        _Row_Address
  B:0090H.0       PUBLIC        OLED_SCL
  C:426EH         PUBLIC        _Delay
  C:42DBH         PUBLIC        _Set_Row_Address
  C:40B7H         PUBLIC        _OLED_DrawBMP
BL51 BANKED LINKER/LOCATER V6.22                                                      04/19/2018  15:13:34  PAGE 5


  -------         PROC          _DELAY
  D:0006H         SYMBOL        Data
  -------         DO            
  D:0004H         SYMBOL        temp
  -------         ENDDO         
  C:426EH         LINE#         45
  C:426EH         LINE#         46
  C:426EH         LINE#         48
  C:4277H         LINE#         49
  C:4277H         LINE#         50
  C:4284H         LINE#         51
  C:428BH         LINE#         52
  -------         ENDPROC       _DELAY
  C:4205H         SYMBOL        L?0120
  -------         PROC          L?0119
  -------         ENDPROC       L?0119
  C:4205H         SYMBOL        L?0120
  -------         PROC          _WRITE_REGISTER
  D:0007H         SYMBOL        Data
  -------         DO            
  D:0006H         SYMBOL        i
  -------         ENDDO         
  C:420AH         LINE#         56
  C:420AH         LINE#         57
  C:420AH         LINE#         60
  C:420CH         LINE#         61
  C:420EH         LINE#         62
  C:4210H         LINE#         63
  C:4210H         LINE#         64
  C:4212H         LINE#         65
  C:4216H         LINE#         66
  C:4216H         LINE#         67
  C:4218H         LINE#         68
  C:421AH         LINE#         70
  C:421AH         LINE#         71
  C:421CH         LINE#         72
  C:421CH         LINE#         73
  C:4220H         LINE#         74
  C:4222H         LINE#         75
  C:4226H         LINE#         76
  C:4228H         LINE#         77
  C:422AH         LINE#         78
  -------         ENDPROC       _WRITE_REGISTER
  -------         PROC          _WRITE_PARAMETER
  D:0007H         SYMBOL        Data
  -------         DO            
  D:0006H         SYMBOL        i
  -------         ENDDO         
  C:424DH         LINE#         80
  C:424DH         LINE#         81
  C:424DH         LINE#         84
  C:424FH         LINE#         85
  C:4251H         LINE#         86
  C:4253H         LINE#         87
  C:4253H         LINE#         88
  C:4255H         LINE#         89
  C:4259H         LINE#         90
BL51 BANKED LINKER/LOCATER V6.22                                                      04/19/2018  15:13:34  PAGE 6


  C:4259H         LINE#         91
  C:425BH         LINE#         93
  C:425DH         LINE#         95
  C:425DH         LINE#         96
  C:425FH         LINE#         97
  C:425FH         LINE#         98
  C:4263H         LINE#         99
  C:4265H         LINE#         100
  C:4269H         LINE#         101
  C:426BH         LINE#         102
  C:426DH         LINE#         103
  -------         ENDPROC       _WRITE_PARAMETER
  -------         PROC          _COLUMN_ADDRESS
  D:0004H         SYMBOL        a
  D:0005H         SYMBOL        b
  C:42A4H         LINE#         111
  C:42A6H         LINE#         112
  C:42A6H         LINE#         113
  C:42ABH         LINE#         114
  C:42B2H         LINE#         115
  -------         ENDPROC       _COLUMN_ADDRESS
  -------         PROC          _ROW_ADDRESS
  D:0004H         SYMBOL        a
  D:0005H         SYMBOL        b
  C:42B9H         LINE#         124
  C:42BBH         LINE#         125
  C:42BBH         LINE#         126
  C:42C0H         LINE#         127
  C:42C5H         LINE#         128
  -------         ENDPROC       _ROW_ADDRESS
  -------         PROC          _CLEARLED
  D:0009H         SYMBOL        color
  -------         DO            
  D:0005H         SYMBOL        j
  D:0004H         SYMBOL        i
  -------         ENDDO         
  C:422BH         LINE#         136
  C:422DH         LINE#         137
  C:422DH         LINE#         140
  C:4234H         LINE#         142
  C:423BH         LINE#         143
  C:423DH         LINE#         144
  C:423DH         LINE#         145
  C:423FH         LINE#         146
  C:423FH         LINE#         147
  C:4244H         LINE#         148
  C:4248H         LINE#         149
  C:424CH         LINE#         150
  -------         ENDPROC       _CLEARLED
  -------         PROC          RAINBOW
  -------         DO            
  D:0005H         SYMBOL        j
  D:0004H         SYMBOL        i
  -------         ENDDO         
  C:41DBH         LINE#         151
  C:41DBH         LINE#         152
  C:41DBH         LINE#         155
BL51 BANKED LINKER/LOCATER V6.22                                                      04/19/2018  15:13:34  PAGE 7


  C:41E2H         LINE#         157
  C:41E9H         LINE#         158
  C:41EBH         LINE#         159
  C:41EBH         LINE#         160
  C:41EDH         LINE#         161
  C:41EDH         LINE#         162
  C:41FCH         LINE#         163
  C:4200H         LINE#         164
  C:4204H         LINE#         165
  -------         ENDPROC       RAINBOW
  -------         PROC          _SET_COLUME_ADDRESS
  D:0004H         SYMBOL        Addr1
  D:0005H         SYMBOL        Addr2
  C:42CAH         LINE#         167
  C:42CCH         LINE#         168
  C:42CCH         LINE#         169
  C:42D1H         LINE#         170
  C:42D6H         LINE#         171
  -------         ENDPROC       _SET_COLUME_ADDRESS
  -------         PROC          _SET_ROW_ADDRESS
  D:0004H         SYMBOL        Addr1
  D:0005H         SYMBOL        Addr2
  C:42DBH         LINE#         175
  C:42DDH         LINE#         176
  C:42DDH         LINE#         177
  C:42E2H         LINE#         178
  C:42E7H         LINE#         179
  -------         ENDPROC       _SET_ROW_ADDRESS
  -------         PROC          _OLED_SHOWCHAR
  D:000FH         SYMBOL        x
  D:0010H         SYMBOL        y
  D:0003H         SYMBOL        chr
  -------         DO            
  D:0011H         SYMBOL        c
  D:0002H         SYMBOL        i
  D:0005H         SYMBOL        j
  D:0012H         SYMBOL        Data1
  D:0013H         SYMBOL        Data2
  D:0001H         SYMBOL        DATA1
  -------         ENDDO         
  C:3C0DH         LINE#         183
  C:3C11H         LINE#         184
  C:3C15H         LINE#         187
  C:3C16H         LINE#         188
  C:3C1BH         LINE#         189
  C:3C23H         LINE#         191
  C:3C2DH         LINE#         193
  C:3C2FH         LINE#         194
  C:3C2FH         LINE#         195
  C:3C51H         LINE#         196
  C:3C73H         LINE#         197
  C:3C75H         LINE#         198
  C:3C75H         LINE#         199
  C:3C8FH         LINE#         200
  C:3C8FH         LINE#         201
  C:3C91H         LINE#         202
  C:3C93H         LINE#         203
BL51 BANKED LINKER/LOCATER V6.22                                                      04/19/2018  15:13:34  PAGE 8


  C:3C95H         LINE#         204
  C:3CAFH         LINE#         205
  C:3CAFH         LINE#         206
  C:3CB2H         LINE#         207
  C:3CB2H         LINE#         208
  C:3CB7H         LINE#         209
  C:3CB9H         LINE#         210
  C:3CBDH         LINE#         211
  C:3CC6H         LINE#         215
  C:3CD0H         LINE#         216
  C:3CDDH         LINE#         217
  C:3CDFH         LINE#         218
  C:3CDFH         LINE#         219
  C:3D01H         LINE#         220
  C:3D23H         LINE#         221
  C:3D25H         LINE#         222
  C:3D25H         LINE#         223
  C:3D3FH         LINE#         224
  C:3D3FH         LINE#         225
  C:3D41H         LINE#         226
  C:3D43H         LINE#         227
  C:3D45H         LINE#         228
  C:3D5FH         LINE#         229
  C:3D5FH         LINE#         230
  C:3D62H         LINE#         231
  C:3D62H         LINE#         232
  C:3D67H         LINE#         233
  C:3D69H         LINE#         234
  C:3D6DH         LINE#         235
  C:3D76H         LINE#         236
  -------         ENDPROC       _OLED_SHOWCHAR
  -------         PROC          _OLED_SHOWSTRING
  D:0009H         SYMBOL        x
  D:000AH         SYMBOL        y
  D:000BH         SYMBOL        chr
  -------         DO            
  D:000EH         SYMBOL        j
  -------         ENDDO         
  C:41AAH         LINE#         239
  C:41B4H         LINE#         240
  C:41B4H         LINE#         241
  C:41B7H         LINE#         242
  C:41C9H         LINE#         243
  C:41D0H         LINE#         244
  C:41D6H         LINE#         246
  C:41D8H         LINE#         247
  C:41DAH         LINE#         248
  -------         ENDPROC       _OLED_SHOWSTRING
  -------         PROC          _OLED_POW
  D:001DH         SYMBOL        m
  D:0001H         SYMBOL        n
  -------         DO            
  D:0006H         SYMBOL        result
  -------         ENDDO         
  C:428CH         LINE#         251
  C:4290H         LINE#         252
  C:4290H         LINE#         253
BL51 BANKED LINKER/LOCATER V6.22                                                      04/19/2018  15:13:34  PAGE 9


  C:4294H         LINE#         254
  C:42A3H         LINE#         255
  C:42A3H         LINE#         256
  -------         ENDPROC       _OLED_POW
  -------         PROC          _OLED_SHOWNUM
  D:0014H         SYMBOL        x
  D:0015H         SYMBOL        y
  D:0016H         SYMBOL        num
  D:0018H         SYMBOL        len
  D:0019H         SYMBOL        size
  -------         DO            
  D:001AH         SYMBOL        t
  D:001BH         SYMBOL        temp
  D:001CH         SYMBOL        enshow
  -------         ENDDO         
  C:4135H         LINE#         263
  C:413DH         LINE#         264
  C:413DH         LINE#         266
  C:4140H         LINE#         267
  C:4149H         LINE#         268
  C:4149H         LINE#         269
  C:416BH         LINE#         270
  C:4179H         LINE#         271
  C:4179H         LINE#         272
  C:417DH         LINE#         273
  C:417DH         LINE#         274
  C:418DH         LINE#         275
  C:418FH         LINE#         276
  C:4192H         LINE#         278
  C:4192H         LINE#         279
  C:41A5H         LINE#         280
  C:41A9H         LINE#         281
  -------         ENDPROC       _OLED_SHOWNUM
  -------         PROC          _OLED_SHOWCHINESE
  D:0009H         SYMBOL        x
  D:000AH         SYMBOL        y
  D:000BH         SYMBOL        no
  -------         DO            
  D:0003H         SYMBOL        i
  D:000CH         SYMBOL        j
  D:000DH         SYMBOL        Data1
  D:000EH         SYMBOL        Data2
  D:000FH         SYMBOL        DATA1
  -------         ENDDO         
  C:3D77H         LINE#         284
  C:3D7DH         LINE#         285
  C:3D7FH         LINE#         288
  C:3D81H         LINE#         290
  C:3D89H         LINE#         292
  C:3D93H         LINE#         294
  C:3D96H         LINE#         295
  C:3D96H         LINE#         296
  C:3DB2H         LINE#         297
  C:3DCEH         LINE#         298
  C:3DD0H         LINE#         299
  C:3DD0H         LINE#         300
  C:3DE6H         LINE#         301
BL51 BANKED LINKER/LOCATER V6.22                                                      04/19/2018  15:13:34  PAGE 10


  C:3DE6H         LINE#         302
  C:3DE9H         LINE#         303
  C:3DEBH         LINE#         304
  C:3DEEH         LINE#         305
  C:3E04H         LINE#         306
  C:3E04H         LINE#         307
  C:3E07H         LINE#         308
  C:3E07H         LINE#         309
  C:3E0CH         LINE#         310
  C:3E0FH         LINE#         311
  C:3E13H         LINE#         312
  C:3E1FH         LINE#         316
  C:3E29H         LINE#         317
  C:3E36H         LINE#         319
  C:3E39H         LINE#         320
  C:3E39H         LINE#         321
  C:3E55H         LINE#         322
  C:3E71H         LINE#         323
  C:3E73H         LINE#         324
  C:3E73H         LINE#         325
  C:3E89H         LINE#         326
  C:3E89H         LINE#         327
  C:3E8CH         LINE#         328
  C:3E8EH         LINE#         329
  C:3E91H         LINE#         330
  C:3EA7H         LINE#         331
  C:3EA7H         LINE#         332
  C:3EAAH         LINE#         333
  C:3EAAH         LINE#         334
  C:3EAFH         LINE#         335
  C:3EB2H         LINE#         336
  C:3EB6H         LINE#         337
  C:3EC2H         LINE#         338
  -------         ENDPROC       _OLED_SHOWCHINESE
  -------         PROC          _OLED_DRAWBMP
  D:0009H         SYMBOL        x1
  D:000AH         SYMBOL        y1
  D:000BH         SYMBOL        x2
  D:000CH         SYMBOL        y2
  D:000DH         SYMBOL        BMP
  -------         DO            
  D:0010H         SYMBOL        i
  D:0011H         SYMBOL        m
  D:0012H         SYMBOL        k
  -------         ENDDO         
  C:40B7H         LINE#         340
  C:40BDH         LINE#         341
  C:40BDH         LINE#         342
  C:40C0H         LINE#         343
  C:40C4H         LINE#         345
  C:40C9H         LINE#         347
  C:40D0H         LINE#         349
  C:40F0H         LINE#         350
  C:40F0H         LINE#         351
  C:4110H         LINE#         352
  C:4110H         LINE#         354
  C:412CH         LINE#         356
BL51 BANKED LINKER/LOCATER V6.22                                                      04/19/2018  15:13:34  PAGE 11


  C:4130H         LINE#         358
  C:4134H         LINE#         359
  -------         ENDPROC       _OLED_DRAWBMP
  -------         PROC          OPEN_DC_POWER
  C:42F8H         LINE#         361
  C:42F8H         LINE#         362
  C:42F8H         LINE#         363
  C:42FAH         LINE#         364
  C:42FDH         LINE#         365
  -------         ENDPROC       OPEN_DC_POWER
  -------         PROC          OFF_DC_POWER
  C:4302H         LINE#         367
  C:4302H         LINE#         368
  C:4302H         LINE#         369
  C:4304H         LINE#         370
  C:4307H         LINE#         371
  -------         ENDPROC       OFF_DC_POWER
  -------         PROC          INITIAL_SSD1327
  C:401BH         LINE#         373
  C:401BH         LINE#         374
  C:401BH         LINE#         376
  C:401DH         LINE#         377
  C:4024H         LINE#         378
  C:4026H         LINE#         380
  C:402BH         LINE#         381
  C:4030H         LINE#         382
  C:4035H         LINE#         383
  C:403AH         LINE#         384
  C:403FH         LINE#         385
  C:4044H         LINE#         386
  C:4049H         LINE#         387
  C:404EH         LINE#         388
  C:4053H         LINE#         389
  C:4058H         LINE#         390
  C:405DH         LINE#         391
  C:4062H         LINE#         392
  C:4067H         LINE#         393
  C:406CH         LINE#         394
  C:4071H         LINE#         395
  C:4076H         LINE#         396
  C:407BH         LINE#         397
  C:4080H         LINE#         398
  C:4082H         LINE#         399
  C:4085H         LINE#         400
  C:408AH         LINE#         401
  C:408FH         LINE#         402
  C:4094H         LINE#         403
  C:4099H         LINE#         404
  C:409EH         LINE#         405
  C:40A3H         LINE#         406
  C:40A8H         LINE#         407
  C:40ADH         LINE#         408
  C:40B2H         LINE#         409
  -------         ENDPROC       INITIAL_SSD1327
  -------         ENDMOD        OLED

  -------         MODULE        ?C?CLDOPTR
BL51 BANKED LINKER/LOCATER V6.22                                                      04/19/2018  15:13:34  PAGE 12


  C:3F7BH         PUBLIC        ?C?CLDOPTR
  -------         ENDMOD        ?C?CLDOPTR

  -------         MODULE        ?C?IMUL
  C:3FA8H         PUBLIC        ?C?IMUL
  -------         ENDMOD        ?C?IMUL

  -------         MODULE        ?C?UIDIV
  C:3FBAH         PUBLIC        ?C?UIDIV
  -------         ENDMOD        ?C?UIDIV

  -------         MODULE        ?C?OFFXADD
  C:400FH         PUBLIC        ?C?OFFXADD
  -------         ENDMOD        ?C?OFFXADD

*** WARNING L16: UNCALLED SEGMENT, IGNORED FOR OVERLAY PROCESS
    SEGMENT: ?PR?_COLUMN_ADDRESS?OLED

*** WARNING L16: UNCALLED SEGMENT, IGNORED FOR OVERLAY PROCESS
    SEGMENT: ?PR?_ROW_ADDRESS?OLED

*** WARNING L16: UNCALLED SEGMENT, IGNORED FOR OVERLAY PROCESS
    SEGMENT: ?PR?_OLED_SHOWNUM?OLED

*** WARNING L16: UNCALLED SEGMENT, IGNORED FOR OVERLAY PROCESS
    SEGMENT: ?PR?OFF_DC_POWER?OLED

Program Size: data=31.0 xdata=0 code=17164
LINK/LOCATE RUN COMPLETE.  4 WARNING(S),  0 ERROR(S)
